:020000040000FA
:02000000A22933
:08000800A2298207C034F9347B
:10001000A434B034993492348234F8348034903437
:1000200087348207D534C134FD3411342934633424
:10003000E93439344D3457346F34820762346234D2
:1000400062346334633463346234633463346334FA
:100050006334100882070800342839283E284228D3
:1000600047284C2850285428170893004D21900AFF
:100070000800C4305A2102309007080000305A218D
:10008000900A0800130811205A21900A080013084A
:100090001D205A21900A080064305A21900A080055
:1000A00000305A21900A08007521900117081302A8
:1000B000031D900A080015088207080071286128AE
:1000C0007A28851D6A281E081902031D08000130C0
:1000D000950008004221D33019079E000330950097
:1000E00008008A2184219B21383019079E000230A4
:1000F0009500080085198028D33019079E00080054
:100100001E081902031D08002C210130950008006B
:100110000D088207A828AB28B228B228AF28B22839
:10012000B228AF28B228B228AF28B228B228AF2808
:10013000B228B228AF28B228B228AF28B228B228F5
:10014000AF28B228B228AF28B228B228B4280800B5
:10015000051D8D0A0800051DB2288D010800051D2A
:1001600003148E0C8D0A0800051DBB2894140E097B
:100170008F008D0108000C158D01080014089410E3
:10018000820708000800C528D2280F08DF39463A40
:100190000319D028153A031D080095219401080081
:1001A000940A080030300F02031CCE28093C031CBF
:1001B000CE2830300F029700950184219B219401B5
:1001C00008000C080C1182070800FD280F29A2293D
:1001D000EC28F9280B29A22995018A2121218421C3
:1001E0009B21B43018079C000E3019079D008C0A23
:1001F0000800B43018079C0001291C0818020319D4
:1002000009291D081902031D08002C2195218C0ABB
:1002100008008C010800B43018079C0008001C0876
:10022000180203198C0108001A081802031D08009F
:100230001B081902031D0800960108001608850610
:1002400008002B3018079A0000300318013E1907E8
:100250009B00103096000800A53018079A00043063
:100260000318013E19079B00103096000800153056
:1002700018079A000E300318013E19079B00103032
:10028000960008002B3018079A001C300318013E16
:1002900019079B001030960008000C30831685006B
:1002A000831285140000051400008510000005105D
:1002B0000000080092000C3083168500831208307D
:1002C0009100920D8514031C851000000514000098
:1002D00005100000910B61290E30831685008312F2
:1002E000051400000510000008000C30831685007E
:1002F00083128510000005140000851400000F30E3
:1003000083168500831208009008031D0800013041
:1003100090000800970A00301702031C9229093C3C
:10032000031808000030970008009508031D080016
:100330000130950008001708052086009508031D68
:100340008613080083168601EF308500C1308100D6
:1003500083128601950194018C018D019001960113
:10036000990198013721051DCA2909309700842178
:10037000952196080319D1290B1DBC29BC30810099
:100380000B1164001E2129201421980A031DB9298C
:10039000990AB9290A3097009B2184211D308D00CC
:1003A000D1290B1DD129BC3081000B1164001E2105
:1003B000882029205B20E120BE201421980A031DFB
:0603C000D129990AD129A0
:02400E00FD3F74
:00000001FF
